:020000040000FA
:100000005C2004201720012883200230A200221443
:100010006B2083200730A600502083200730A600E5
:10002000502083200F30A60050204B200800832052
:100030000230A2001D30A60022146B202708A60063
:100040005020832022106B2032203A208320260863
:10005000A3003F2032203A2083202608A400452018
:100060004B20080080208C118320911580208C1D4E
:1000700037280800802013088320A600080083206A
:1000800091121116111A4228080083209116111698
:10009000111A482808008320111511194D2808004D
:1000A00080208C1183202608802093008C1D5628E8
:1000B0008320111B59280800832086019417802073
:1000C000283094008320093093008715071680207C
:1000D0008715071608008320111411186D28802039
:1000E0008C11000083202208802093008C1D76282C
:1000F0008320111F0800911491187C286F28080094
:1001000003138312080003138316080003178312D6
:08011000080003178316080024
:02400E00F13F80
:00000001FF
